:100000000C9438000C9423051895000018950000F6
:10001000189500001895000018950000189500002C
:10002000189500001895000018950000189500001C
:100030001895000018950000189500000C943A05DA
:10004000189500000C948A06189500001895000079
:1000500018950000189500001895000018950000EC
:1000600018950000189500001895000018950000DC
:100070008FEF8DBFC0EEE8ED4E2E84E08EBFD4E052
:10008000F4E05F2EEEEFF3E0A0E0B1E0A89584B7D6
:10009000082E877F84BF88E1992781BD91BD88277D
:1000A0008D933197E9F70E94A20666248FEF8ABBF1
:1000B00080E08BBB81EE87BB8FE188BB8FEF84BB79
:1000C0008FEF85BB8BEF81BB8FEF82BB8FEF86B944
:1000D0008FEF87B980E08FBD82E08EBD89B78068E1
:1000E00089BF85B78C7F85BF8BB780648BBF7894C1
:1000F00006B34EE10423A3E0B1E00C9391E0A3E04A
:10010000B1E00E94920780E08093290180E0809313
:100110002C0180E08093250180E080932D010091E7
:100120002901003081E009F080E08F9300912C01DB
:10013000003081E009F080E09F9189238F93009146
:100140002501003081E009F080E09F9189238F93A1
:1001500000912D01003081E009F080E09F9189231A
:10016000882311F40C94B700C09A0C94B800C0987E
:1001700083E08093350182E38093360184B7877FE3
:1001800084BF8FE181BD87E081BD81B5886081BD7D
:100190000027A2E0B1E08C9187FB0EF401E041E082
:1001A000041711F00C94910100910101003011F03D
:1001B0000C94890100910001003111F00C94E600CB
:1001C00080912D0191E0892780932D0100910001FC
:1001D000013111F00C94F20080912D0192E08927F9
:1001E00080932D0100910001063011F00C94FB006A
:1001F00080E080932C0100910001033011F00C94F9
:10020000040182E380932C0100910001043011F07D
:100210000C94180100912901053018F011F00C948C
:1002200013010C94180180912901815080932901B8
:1002300000910001013011F00C943201009129016C
:10024000023310F00C942901A9E2B1E08C918F5F88
:100250008C9300912901053010F00C94320185E057
:100260008093290100910001073011F00C943B01AB
:1002700080E080932901009100010D3011F00C9471
:10028000440182E38093290100910001023011F0C2
:100290000C944D0181E0809325010091000105300F
:1002A00011F00C94560182E0809325010091000129
:1002B000083011F00C945F0183E0809325010091D8
:1002C0000001003011F00C94680184E08093250156
:1002D000009100010F3011F00C94710180E08093C7
:1002E0002501009100010C3011F00C94830180E095
:1002F0008093290180E080932C0180E08093250188
:1003000080E080932D01C79A84E190E00E94070766
:10031000C798809102018F77809302018BB7806428
:100320008BBF0027A2E0B1E08C9186FB0EF401E0C8
:1003300041E0041711F00C945003809102018F7B6F
:1003400080930201A89581E08093300100913001F3
:10035000083018F011F00C942A02A0E3B1E0AD903F
:10036000BB24ABE1B1E0AA0DBB1D4C91A0E3B1E011
:10037000AD90BB24A3E1B1E0AA0DBB1D0C91041705
:1003800018F011F00C94C6010C94D001A0E3B1E078
:10039000AD90BB24A3E1B1E0AA0DBB1D0E9497065E
:1003A000A0E3B1E0AD90BB24ABE1B1E0AA0DBB1D71
:1003B0004C91A0E3B1E0AD90BB24A3E1B1E0AA0D64
:1003C000BB1D0C91041710F00C94F101A0E3B1E0F7
:1003D000AD90BB24A3E1B1E0AA0DBB1D8C918F5F52
:1003E0008C93A0E3B1E0AD90BB24A3E1B1E0AA0DF2
:1003F000BB1D0D911127A0E3B1E0AD90BB24A3E19B
:10040000B1E0AA0DBB1D4D9155270E948807A3E3BB
:10041000B1E00D931C93A3E3B1E00D911C9149E170
:1004200050E00E94E406A3E3B1E04D935C93809119
:100430003301A0E3B1E0AD90BB24ABE0B1E0AA0D85
:10044000BB1D8C93A0E3B1E08C918F5F8C9310F473
:100450000C94A6014091290100912801041718F07D
:1004600011F00C9435020C943A02809128018150CD
:10047000809328014091290100912801041710F070
:100480000C944702A8E2B1E08C918F5F8C93A8E2B4
:10049000B1E00D911127A8E2B1E04D9155270E94DE
:1004A0008807A3E3B1E00D931C93A3E3B1E00D91A2
:1004B0001C9149E150E00E94E406A3E3B1E04D93B2
:1004C0005C93809133018093270140912C0100912E
:1004D0002B01041718F011F00C9470020C947502A3
:1004E00080912B01815080932B0140912C01009130
:1004F0002B01041710F00C948202ABE2B1E08C9156
:100500008F5F8C93ABE2B1E00D911127ABE2B1E0CC
:100510004D9155270E948807A3E3B1E00D931C93EA
:10052000A3E3B1E00D911C9149E150E00E94E40683
:10053000A3E3B1E04D935C938091330180932A0152
:1005400006B34EE10423A4E0B1E00C9391E0A4E0F3
:10055000B1E00E9492074091030100910401041749
:1005600081E009F480E08F9340910401009105013E
:10057000041781E009F080E09F918923882311F41A
:100580000C944903A6E0B1E08C918F5F8C930091AD
:100590000601043011F00C944703A4E0B1E00C9183
:1005A00000FB00270EF401E0A3E0B1E08C9180FB9A
:1005B00044270EF441E0041711F40C94ED0200916D
:1005C0002501003011F00C94EA0281E080932501AE
:1005D0000C94ED0280E080932501A4E0B1E00C9141
:1005E00001FB00270EF401E0A3E0B1E08C9181FB58
:1005F00044270EF441E0041711F40C940D0300910C
:100600002901003011F00C940A0382E38093290140
:100610000C940D0380E080932901A4E0B1E00C91DB
:1006200002FB00270EF401E0A3E0B1E08C9182FB15
:1006300044270EF441E0041711F40C942503809133
:100640002D0191E0892780932D01A4E0B1E00C9168
:1006500003FB00270EF401E0A3E0B1E08C9183FBE3
:1006600044270EF441E0041711F40C943D038091EB
:100670002D0192E0892780932D01809104018093C0
:100680000301C79A84E190E00E940707C7980C9481
:100690005003809104018093050180E0809306015E
:1006A0000027A2E0B1E08C9185FB0EF401E041E06F
:1006B000041711F00C94DF03809102018F7D809369
:1006C0000201ADE2B1E00C9100FB00270EF401E065
:1006D00041E0041711F00C947A0300912E010630CA
:1006E00010F00C947803AEE2B1E08C918F5F8C93A4
:1006F0000C94880300912E01003018F011F00C9436
:1007000083030C94880380912E01815080932E01E5
:10071000ADE2B1E00C9101FB00270EF401E041E0F5
:10072000041711F00C94A10300912F01063010F072
:100730000C949F03AFE2B1E08C918F5F8C930C948B
:10074000AF0300912F01003018F011F00C94AA03B0
:100750000C94AF0380912F01815080932F01ECEF17
:10076000FCE0AEE2B1E08C919927A1E3B1E00E94F8
:10077000AA0702B34FE00423A2E3B1E00C93009177
:10078000310140913201042B02BBE4E0FDE0AEE216
:10079000B1E08C919927A1E3B1E00E94AA07ECE0B7
:1007A000FDE0AFE2B1E08C919927A2E3B1E00E94B5
:1007B000AA070091310140913201042B05BB0027AB
:1007C000A2E0B1E08C9184FB0EF401E041E004175B
:1007D00011F00C941F05809102018F7E809302011D
:1007E00000912901003081E009F080E08F930091B1
:1007F0002C01003081E009F080E09F9189238F93E4
:1008000000912501003081E009F080E09F9189236B
:100810008F9300912D01003081E009F080E09F91DD
:100820008923882311F40C941804C09A0C94190499
:10083000C09800912501003011F00C943704A6E215
:10084000B1E08C918F5F8C9300912601093011F0FB
:100850000C942D0481E08093260180E0A6E2B1E0B3
:10086000AD90BB24ABE1B1E0AA0DBB1D8C93009110
:100870002501013011F00C947204A6E2B1E08C91D4
:100880008F5F8C9300912601093011F00C944B047A
:1008900081E08093260140913601A6E2B1E0AD905F
:1008A000BB24ABE1B1E0AA0DBB1D0C91041711F400
:1008B0000C94670480913601A6E2B1E0AD90BB24B0
:1008C000ABE1B1E0AA0DBB1D8C930C947204809136
:1008D0003501A6E2B1E0AD90BB24ABE1B1E0AA0DD9
:1008E000BB1D8C9300912501023011F00C94AC04D7
:1008F000A6E2B1E08C918F5F8C93009126010930C4
:1009000011F00C94860481E0809326010091360159
:1009100040913501041BA1E3B1E00C93A1E3B1E0E8
:100920008C9199278A939A930E94A906A1E3B1E03A
:100930000C930091310140913501040FA1E3B1E026
:100940000C9380913101A6E2B1E0AD90BB24ABE104
:10095000B1E0AA0DBB1D8C9300912501033011F06D
:100960000C9401058AEF90E08A939A930E94A9065D
:10097000A1E3B1E00C930091310148E00E94AD0782
:10098000A6E2B1E08C93A1E3B1E00C9148E00E94B3
:10099000AD070C93A1E3B1E00C9143E00E94AD07D9
:1009A0008C9300913101003011F00C94E10480E04F
:1009B000A6E2B1E0AD90BB24ACE1B1E0AA0DBB1D55
:1009C0008C9300913101013011F00C94F10489E114
:1009D000A6E2B1E0AD90BB24ACE1B1E0AA0DBB1D35
:1009E0008C9300913101023011F00C94010582E3E7
:1009F000A6E2B1E0AD90BB24ACE1B1E0AA0DBB1D15
:100A00008C9300912501043011F00C941F05A6E28F
:100A1000B1E08C918F5F8C9300912601093011F029
:100A20000C94150581E08093260182E3A6E2B1E0F3
:100A3000AD90BB24ABE1B1E0AA0DBB1D8C930C942F
:100A4000C800F894FFCF8BB78F7B8BBF78940E9440
:100A50001607A1E0B1E02C93A0E0B1E01C93A0E068
:100A6000B1E08C918F778C938091020180688093A4
:100A7000020118950F921F922F923F924F925F9210
:100A80007F92AF92BF920F931F932F933F934F93F9
:100A90005F936F937F938F939F93AF93BF93CF9306
:100AA000DF93EF93FF938FB78F9386E09FEF9DBD0A
:100AB0008CBDABE0B1E08C918F5F8C9300910B010A
:100AC000043611F00C94670580E080930B0140918F
:100AD0000C0100910B01041710F00C947605809125
:100AE00024018160809324010C947B058091240172
:100AF0008E7F8093240140910D0100910B0104171A
:100B000010F00C948A058091240182608093240166
:100B10000C948F05809124018D7F80932401409156
:100B20000E0100910B01041710F00C949E058091AA
:100B300024018460809324010C94A30580912401F6
:100B40008B7F8093240140910F0100910B010417CA
:100B500010F00C94B20580912401886080932401E8
:100B60000C94B70580912401877F809324014091E4
:100B7000100100910B01041710F00C94C605809130
:100B800024018061809324010C94CB058091240181
:100B90008F7E809324014091110100910B01041775
:100BA00010F00C94DA058091240180628093240176
:100BB0000C94DF05809124018F7D80932401409166
:100BC000120100910B01041710F00C94EE058091B6
:100BD00024018064809324010C94F3058091240106
:100BE0008F7B809324014091130100910B01041726
:100BF00010F00C94020680912401806880932401F7
:100C00000C940706809124018F77809324014091F2
:100C1000270100910B01041710F00C941206C69ADC
:100C20000C941306C69840912A0100910B010417F9
:100C300010F00C941E06C59A0C941F06C598A4E2E9
:100C4000B1E08C918BBBA7E0B1E00E949B06A7E0CE
:100C5000B1E00D911C91003951E0150711F00C9491
:100C6000620680E090E0A7E0B1E08D939C938091D4
:100C70000201806480930201A9E0B1E08C918F5F52
:100C80008C9300910901023011F00C94620680E00F
:100C90008093090180910201806280930201AAE0A1
:100CA000B1E08C918F5F8C9300910A01053011F0B7
:100CB0000C94620680E080930A01809102018061B9
:100CC000809302018F918FBFFF91EF91DF91CF91C0
:100CD000BF91AF919F918F917F916F915F914F9154
:100CE0003F912F911F910F91BF90AF907F905F9098
:100CF0004F903F902F901F900F901895F0703010EC
:100D0000000000000303030303020000FCF8F0E00E
:100D1000C08000008F939F938FB73395539509F44C
:100D2000439591E892BF9F918FBF8F9118958C91B9
:100D300081508C930895ED91FC91EF5FFF4FFC93F0
:100D4000EE93089515E000E0009337011093380109
:100D5000089540913701509138010DEF13E40E943E
:100D6000BE060D53114640E050E82ED000933701E7
:100D7000109338015991499127D0089509D00E94C4
:100D8000880700FC10D0089503D01ED001F8F9CFD9
:100D90000024E89457FF02C009D0689400F80BD0F3
:100DA00010F80124089502D009D008955095409577
:100DB0004F5F5F4F0895E89417FF089500951095D1
:100DC0000F5F1F4F68940895352F242FE894452B0B
:100DD00011F468940895512F402F0027112780E1C6
:100DE000440F551F001F111F021B130B416018F405
:100DF000020F131F4E7F8A9599F708953197F1F7E7
:100E00000895689462F80895E89462F80895EF935D
:100E1000FF93EE27E82BE92B31F0E0EAFFE0319772
:100E2000F1F70197D1F7FF91EF9108950F933F9359
:100E30004F935F932F923F928F939F938FB78F9390
:100E400083B78F93826083BF89B78F93826089BF96
:100E500081E882BF552744273327403D08F047C02B
:100E6000373324F4829BF8CFF8CF41C04830ECF7F9
:100E70008299FCCF33273232D4F5829BFCCF932F5B
:100E8000332711272227913110F0969511E0292E52
:100E90002694322C290E990F390E113021F032157B
:100EA00034F58299FCCF33270CE03215F0F38299A8
:100EB00009C08894111F221F3315CCF4829BFCCFEC
:100EC000332708C00894111F221F331584F4829918
:100ED000FCCF33270A9549F7912F991F221F991F9D
:100EE000221F25FB17F926FB16F92F7102C01FEFF1
:100EF0002FEF8F9189BF8F9183BF8F918FBF9F916C
:100F00008F913F902F905F914F913F910F91089556
:100F10000F92B801469F8001479F100D569F100DFC
:100F20000F900895903029F08C9186959A95E9F765
:100F30008C930895C89531960020089591E005C0DE
:100F400092E003C094E001C098E0F4DF0D929A951E
:100F5000E1F70895E80FF91FF1CFFF93881BF9E03F
:100F6000001FFA9511F4FF910895881F841B18F44F
:0A0F7000840F8894F5CF0894F3CFA6
:00000001FF
